:02000000952A3F
:10000800FF00030E8301DE000A08DF008A01700882
:10001800A0000B1D1428A80A0319A90A81010B11B5
:100028000B1C7828061A1A2871101B287114051A37
:100038001F28031420280310711C2628031C2628B7
:10004800711427287110711C3128193023020318E4
:100058002F28A30A31280130A300861A35287110E9
:1000680036287114051A3A2803143B280310711C0A
:100078004128031C4128711442287110711C4C2816
:100088002308013C03184A28A3034C281930A3006D
:10009800061F62288030F000803025067002031D9C
:1000A800572824080A3C03185E280A30A402031CB7
:1000B800A50361280130A400A5017728861F7728A9
:1000C80080302506F00080307002031D6D28F53061
:1000D8002402031874280A30A4070318A50A7728ED
:1000E800FF30A400A5010B102008F0005F088A006B
:0A00F8005E0E8300FF0E7F0E09006C
:0E0102008312031322088A00210882000800DD
:10011000831203137008A1007108A20081208A11C4
:100120000A128000840AA10A0319A20AF203031D1D
:040130008E2808000D
:100134000730831203139F00831681120112811565
:10014400011181100110831281018B178B160B1280
:100154008B15103083168500F030860083128501DC
:100164008601A801A9012B3084004930F000043035
:10017400F1000A30F20088200130A300DD017F3055
:06018400A400A501080023
:10018A00831203132308013A031DE2282A080319DC
:10019A00D8282B3084004930F0000430F1000A30AE
:1001AA00F2008820E1282B3084005C30F000043013
:1001BA00F1000930F20088208D2A2308023A031D33
:1001CA00FD282A080319F3282B3084003F30F00059
:1001DA000430F1000A30F2008820FC282B30840019
:1001EA006530F0000430F1000930F20088208D2AD1
:1001FA002308033A031D18292A0803190E292B304C
:10020A008400D230F0000330F1001130F20088206F
:10021A0017292B3084001430F0000430F1000F301D
:10022A00F20088208D2A2308043A031D26292B3040
:10023A008400A930F0000430F1000630F200882072
:10024A008D2A2308053A031D34292B308400AF3048
:10025A00F0000430F1000630F20088208D2A2308CD
:10026A00063A031D4F292A08031945292B30840011
:10027A007730F0000430F1000930F20088204E296E
:10028A002B3084009030F0000430F1000730F20087
:10029A0088208D2A2308073A031D5D292B30840004
:1002AA003130F0000430F1000E30F20088208D2A3F
:1002BA002308083A031D6B292B3084002330F000F1
:1002CA000430F1000E30F20088208D2A2308093A02
:1002DA00031D79292B308400F430F0000330F1003B
:1002EA001030F20088208D2A23080A3A031D872934
:1002FA002B3084000430F0000430F1001030F2009A
:10030A0088208D2A23080B3A031DA2292A080319DB
:10031A0098292B3084006E30F0000430F100093047
:10032A00F2008820A1292B3084008930F0000430A3
:10033A00F1000730F20088208D2A23080C3A031DA9
:10034A00B0292B3084009D30F0000430F1000630D3
:10035A00F20088208D2A23080D3A031DBE292B306E
:10036A008400A330F0000430F1000630F200882047
:10037A008D2A23080E3A031DD9292A080319CF29E1
:10038A002B308400BB30F0000430F1000630F2005C
:10039A008820D8292B308400C430F0000430F100C2
:1003AA000330F20088208D2A23080F3A031DF4290E
:1003BA002A080319EA292B308400B530F0000430EA
:1003CA00F1000630F2008820F3292B308400C13076
:1003DA00F0000430F1000330F20088208D2A23084F
:1003EA00103A031D022A2B3084005830F0000330E3
:1003FA00F1002130F20088208D2A2308113A031DCA
:10040A001D2A2A080319132A2B3084007930F00098
:10041A000330F1001D30F20088201C2A2B308400A2
:10042A009630F0000330F1001930F20088208D2A4E
:10043A002308123A031D2B2A2B3084009730F00030
:10044A000430F1000630F20088208D2A2308133A7E
:10045A00031D392A2B308400AF30F0000330F1003D
:10046A001230F20088208D2A2308143A031D472AE5
:10047A002B3084005330F0000430F1000930F200D0
:10048A0088208D2A2308153A031D552A2B3084000B
:10049A008030F0000430F1000930F20088208D2A03
:1004AA002308163A031D632A2B308400E330F00038
:1004BA000330F1001130F20088208D2A2308173A00
:1004CA00031D712A2B308400C130F0000330F10083
:1004DA001130F20088208D2A2308183A031D7F2A3A
:1004EA002B308400F530F0000230F1003230F20097
:1004FA0088208D2A2308193A031D8D2A2B3084005F
:10050A002730F0000330F1003130F20088208D2AC4
:10051A005D082B3E84000008E0006008F000080037
:10052A009A2080302906F000803025067002031DCB
:10053A00A02A24082802FF30031C0030F0007008AB
:10054A00A60070080319F32A0030051A0130AA0020
:10055A002A08013AFF30031D0030AA002B085D0269
:10056A000318B92ADD0AC62A0130DD002A08031950
:10057A00C62A193023020318C42AA30AC62A01303C
:10058A00A300C5207008A7002718CD2A0510CE2A77
:10059A000514A718D22A8510D32A85142719D72A11
:1005AA000511D82A0515A719DC2A8511DD2A851512
:1005BA00271AE12A0610E22A0614A71AE62A861042
:1005CA00E72A8614271BEB2A0611EC2A0615A71B15
:1005DA00F02A8611F12A8615A801A901962AF42A79
:1005EA003134013401340134013401340134023428
:1005FA00023402340234023402340434043404343B
:10060A00043404340434083408340834083408340C
:10061A0008341034103410341034103410342034A8
:10062A0020342034203420342034403440344034C0
:10063A0040344034403480348034803480348034D0
:04064A0080340034C4
:10064E0030340134003401340034013400340234C7
:10065E0000340234003402340034043400340434E0
:10066E0000340434003408340034083400340834C0
:10067E00003410340034103400341034003420347C
:10068E0000342034003420340034403400344034FC
:10069E0000344034003480340034803400348034EC
:0206AE00003416
:1006B00020348034003480340034403400344034FA
:1006C000003420340034203400341034003410342A
:1006D0000034083400340834003404340034043462
:1006E0000034023400340234003401340034013464
:0206F0000034D4
:1006F2001C34C0340034C03400343034003430345C
:1007020000340C3400340C34003403340034033429
:1007120000340C3400340C340034303400343034BF
:0A0722000034C0340034C034003449
:10072C001834C0340034C034003430340034303425
:10073C0000340C3400340C340034033400340334EF
:10074C0000340C3400340C34003430340034303485
:02075C00003467
:10075E0011348034013440340234203404341034E3
:10076E0008341034083420340434403402348034D5
:04077E00013400340E
:1007820010340134033407340F341F343F347F34C0
:10079200FF34FE34FC34F834F034E034C0348034B6
:0207A200003421
:1007A4001034013402340434083410342034403416
:1007B4008034403420341034083404340234013496
:0207C4000034FF
:1007C60010348034C034E034F034F834FC34FE3471
:1007D600FF347F343F341F340F340734033401347D
:0207E6000034DD
:1007E8000F3400340134043402340834043410342F
:1007F80008342034103440342034803440340034F9
:100808000F340034403480342034403410342034E1
:100818000834103404340834023404340134003405
:100828000E34013402340434083410342034403493
:0E083800803440342034103408340434023448
:100846000D3400340134033407340F341E343C3481
:0C0856007834F034E034C03480340034D6
:100862000D3400348034C034E034F03478343C3415
:0C0872001E340F3407340334013400340A
:10087E0009348034403420341034083404340234C3
:04088E0001340034FD
:10089200093401340234043408341034203440342E
:0408A200803400346A
:1008A600083418343C347E34FF34E734C33481349E
:0208B60000340C
:1008B8000834013402340434083410342034403409
:0208C80080347A
:1008CA000834803440342034103408340434023478
:0208DA000134E7
:1008DC000834C03430340C3403340C343034C03469
:0208EC000034D6
:1008EE0008341834243442348134423424341834D5
:0208FE000034C4
:1009000008348134C334E734FF347E343C34183443
:020910000034B1
:0E0912000634C03430340C3403340C3430342A
:0E0920000634183424344234813442342434F2
:0C092E0005340034FF3400340034003481
:0C093A000534C03430340C340334003475
:0C094600053403340C343034C034003469
:0C0952000534183424344234813400345D
:0C095E0005348134423424341834003451
:0C096A0005345534AA345534AA34003446
:0C09760005340F34F0340F34F03400343A
:0609820002345534AA34D2
:0609880002340F34F034CC
:02400E001A2175
:00000001FF
